:020000040000FA
:0400000072303A28F8
:08000800A000030EA100831209
:1000100005191028831601178312B23081002B288E
:1000200083160113831203140B190310A80DA90DD5
:10003000AA0DAB0DAC0DAC16FF302C02031D2B2806
:10004000FA302B02031D2B2831152A08AF0029088E
:10005000AE002808AD008B100B11210E8300A00EFE
:04006000200E090065
:0C007400203084008001840A6030040207
:10008000031C3C281230B000D5218316FF239000BA
:10009000831283160C308505870183128501870141
:1000A000073099000030831691008312C830831600
:1000B0008100831231309000003083168C0083124F
:1000C00010308B00831600309B001C141A0883121A
:1000D000BC00831610309B001C141A088312BD004C
:1000E000FA2181018E018F010B118B100B108C01F5
:1000F0008B17892031198C20B921B30B8728031065
:1001000085190314B90DF030390203196221FB215E
:10011000792864003210080031110130B7008B13C8
:100120002030370783169B001C141A088312A40082
:100130001030370783169B001C141A088312A30083
:10014000A6000230A6060030370783169B001C1459
:100150001A088312A200A7000130A7068B17321CD1
:10016000B72822090339A200A309A409A509240874
:100170002F02031D5C2923082E02031D0B292208D0
:100180002D02031D5C2901303702031DCC283D18C8
:10019000CC283D143E14E62102303702031DD52839
:1001A000BD18D528BD143E14E92103303702031DC4
:1001B000DE283D19DE283D153E14EA2104303702C1
:1001C000031DE728BD19E728BD153E14EB210530B6
:1001D0003702031DF0283D1AF0283D163E14EC218D
:1001E00006303702031DF928BD1AF928BD163E1442
:1001F000ED2107303702031D02293D1B02293D175F
:100200003E14EE2108303702031D0B29BD1B0B29BC
:10021000BD173E14EF2126082E02031D5C29270876
:100220002D02031D5C2901303702031D1C293D1CD2
:100230001C293D103E14F02102303702031D2529F0
:10024000BD1C2529BD103E14F32103303702031DC8
:100250002E293D1D2E293D113E14F4210430370274
:10026000031D3729BD1D3729BD113E14F521053069
:100270003702031D40293D1E40293D123E14F62140
:1002800006303702031D4929BD1E4929BD123E14FF
:10029000F72107303702031D52293D1F52293D1314
:1002A0003E14F82108303702031D5B29BD1F5B296E
:1002B000BD133E14F9215C29B70A02303702031836
:1002C00008008F280130B600B300B400B500B700B5
:1002D00085018701B1138920B30B88290310851983
:1002E0000314B90DF03039020319AF29B41F850189
:1002F000B41F8701B40B88293708B6080319B60064
:1003000003198629FF3085008700B6039630B400B4
:10031000311D6B293111321C92292D090339AD0091
:10032000AE09AF092F1C6B298E018F010C1C6B29A4
:100330000C102E1E6B298B1320303707BB002F08A3
:10034000BA00C22110303707BB002E08BA00C22104
:1003500000303707BB002D08BA00C2218B1785017A
:100360008701B70AB60102303702031C6B29FA2154
:1003700008003E1C08003E101030BB003D08BA00CB
:10038000C22108008B133A0883161C159A003B08FB
:100390009B0055309D00AA309D009C1464009C1861
:1003A000CE291C1183128B170800FF30D4000230B5
:1003B000D5000C30D600BA30D7003730D800DA304C
:1003C000D9006F30DA00B830DB0008000130BD0022
:1003D00008000800080008000800080008000800DD
:1003E00085018701080008000800080008000800CF
:1003F00008000800080001303D05031908005C18DA
:100400000516DC1885165C190514DC1985145C1AB0
:100410008714DC1A07155C1B0714DC1B87165D1894
:100420000716DD188715E6300E02031C212A051673
:1004300085160514851487140715071487160716E3
:1004400087158F08031908008F018501870154085B
:10045000DE00AE22D4005508DE00AE22D5005608DC
:10046000DE00541CAE22D6005708DE00D41CAE229B
:10047000D7005808DE00541DAE22D8005908DE000F
:10048000D41DAE22D9005A08DE00541EAE22DA0076
:100490005B08DE00D41EAE22DB00CA0B572A5408CC
:1004A000CA00D4185C14D41E5C10D41D5C10CB0B95
:1004B000612A5508CB00D51ADC14551DDC10551FD8
:1004C000DC10CC0B6B2A5608CC00561A5C15561F54
:1004D0005C11D61D5C11CD0B752A5708CD00571A3B
:1004E000DC15D71FDC11D71DDC11CE0B7F2A580875
:1004F000CE00D81B5C16D81F5C12D81C5C12CF0B28
:10050000892A5908CF00591ADC16591EDC12D91F46
:10051000DC12D00B932A5A08D000DA195C17DA1DC6
:100520005C135A1E5C13D10B9D2A5B08D1005B1A29
:10053000DC175B1EDC13DB1FDC13D20BA52A56086D
:10054000D200D51B5D14D71F5D10D30BAD2A570801
:10055000D300D61BDD14D81FDD100800C001DE0853
:100560000319DE035E184014DE1A40144008C0016F
:100570005E1C4014DE1E4014C005C00C5E0C08005A
:084000000F000300020006009E
:02400E00CC01E3
:10420000010078007A007C007E007B0079007F004E
:104210007D007A0078007E007C00FF00FF00FF0038
:104220000000F200F600FA00FE00F200F600FA00CC
:10423000FE00F200F600FA00FE00FF00FF00FF00A3
:10424000010005000500050005000900090009003E
:1042500009000D000D000D000D00FF00FF00FF0024
:10426000FF00FF00FF00FF00FF00FF00FF00FF0056
:10427000FF00FF00FF00FF00FF00FF00FF00FF0046
:10428000FF00FF00FF00FF00FF00FF00FF00FF0036
:10429000FF00FF00FF00FF00FF00FF00FF00FF0026
:1042A000FF00FF00FF00FF00FF00FF00FF00FF0016
:1042B000FF00FF00FF00FF00FF00FF00FF00FF0006
:1042C000FF00FF00FF00FF00FF00FF00FF00FF00F6
:1042D000FF00FF00FF00FF00FF00FF00FF00FF00E6
:1042E000FF00FF00FF00FF00FF00FF00FF00FF00D6
:1042F000FF00FF00FF00FF00FF00FF00FF00DD00E8
:00000001FF
